:1000000000308A00492900008A1D0A128A190A163E
:100010008A11831A0F28A500030EA6001428831244
:10002000A500030EA600A6140A08AD00A50E04083C
:10003000A7002008A8002108A9002208AA00230878
:10004000AB002408AC0083120B1E28288B18502804
:100050008B1E2C280B1952288C308400001C32284F
:100060000C1854288C308400801E38288C1A56288E
:10007000270884002808A0002908A1002A08A20057
:100080002B08A3002C08A4002D088A000A1A8A1540
:100090000A12260E83008312250EA6188316090065
:1000A0008A1134298A119E288A113C298A11F12843
:1000B0000A108A100A1182073F3406345B344F3429
:1000C00066346D347D3407347F346F347734603474
:1000D00066345E3440340034BF348634DB34CF348D
:1000E000E634ED34FD348734FF34EF34F734E03454
:1000F000E634DE34C03480340A108A100A118207D4
:100100000934003403340934063409340934093419
:100110005C08A1015B02031890285B08A0009C28E2
:10012000A0010830DD00DB0DA00D5C0820020318E3
:10013000A000A10DDD0B93288A11A8288501870155
:1001400088018901D50A5508DB000C30DC008828BD
:100150002008D500063055020318C1280130870059
:100160005508A1000319B8280310870DA10BB42866
:100170002E305507840000085820A100210888006F
:10018000EE280A3055020318DA2806305502A1007D
:1001900001308500A1080319D1280310850DA10B9A
:1001A000CD282E305507840000085820A1002108D2
:1001B0008800EE280A305502A10001308900A1080C
:1001C0000319E6280310890DA10BE2282E305507EC
:1001D000840000085820A100210888000B118A1112
:1001E0003828D208031D02290608A000A00E0F30EF
:1001F000A0052008FF3A0739D40054087C20A1004C
:100200002108D30053085207A0003A302007840089
:100210001A088000D20A03305202031D322910103E
:10022000D2013A08C6003B08C7003C08C8003D0898
:10023000C9003E08CA003F08CB004008CC00410876
:10024000CD004208CE004308CF004408D000450846
:10025000D1008316980110309800831298019030D5
:1002600098009A018A1138288F018E011014D2014A
:100270009A018B108A11382898019030980010103C
:100280000930D300D2018316401083120C108A115A
:10029000382884011F3083059F3084000730800098
:1002A000D201D5010930D30083168501FF308600C5
:1002B000C0308700880189019801103098008312AE
:1002C00098019030980081010430A000A01D702991
:1002D00007308101813084000008C0390F38800068
:1002E0006400813084000008C039200480008B162F
:1002F000253090008F018E018130840000130B1691
:100300008C3084008016C0308B0403081839A0009C
:100310001830200203198D29A029F030BA00FF30CF
:10032000BB000F30BC00F030BD00FF30BE000F300E
:10033000BF00F030C000FF30C1000F30C200A12963
:10034000A1293A08C6003B08C7003C08C8003D0880
:10035000C9003E08CA003F08CB004008CC00410855
:10036000CD004208CE004308CF004408D000450825
:10037000D100640046088039D900D90ED90CD90CB7
:10038000D90C0130D90546084039A000A00EA00CB8
:100390000730A0052008D90446082039A000A00C89
:1003A000A00CA00C1F30A0052008D9044608103965
:1003B000A0000310A00C20085904D80046080139F9
:1003C0000038031D581658081F39AE00640047084E
:1003D0000839D900D90CD90CD90C1F30D9054708D8
:1003E0000439A0000310A00C2008D90447080239E2
:1003F000A0000310A00D2008D90447080139A0006F
:10040000A00DA00DA00DF830A00520085904D800BB
:10041000460802390038031D581658081F39AF0026
:10042000640047088039D900D90ED90CD90CD90CF1
:100430000130D90547084039A000A00EA00C0730B4
:10044000A0052008D90447082039A000A00CA00C62
:10045000A00C1F30A0052008D90447081039A000BF
:100460000310A00C20085904D800460804390038AD
:10047000031D581658081F39B00064004808083991
:10048000D900D90CD90CD90C1F30D905480804392A
:10049000A0000310A00C2008D90448080239A000CD
:1004A0000310A00D2008D90448080139A000A00DB0
:1004B000A00DA00DF830A00520085904D80046086A
:1004C00008390038031D581658081F39B100640058
:1004D00049088039D900D90ED90CD90CD90C013072
:1004E000D90549084039A000A00EA00C0730A0058E
:1004F0002008D90449082039A000A00CA00CA00CA9
:100500001F30A0052008D90449081039A0000310A5
:10051000A00C20085904D800490801390038031DEF
:10052000581658081F39B20064004A080839D90023
:10053000D90CD90CD90C1F30D9054A080439A000B0
:100540000310A00C2008D9044A080239A0000310A7
:10055000A00D2008D9044A080139A000A00DA00D63
:10056000A00DF830A00520085904D8004908023928
:100570000038031D581658081F39B30064004A0894
:100580008039D900D90ED90CD90CD90C0130D90534
:100590004A084039A000A00EA00C0730A005200892
:1005A000D9044A082039A000A00CA00CA00C1F30D0
:1005B000A0052008D9044A081039A0000310A00C97
:1005C00020085904D800490804390038031D58167A
:1005D00058081F39B40064004B080839D900D90CF9
:1005E000D90CD90C1F30D9054B080439A0000310D1
:1005F000A00C2008D9044B080239A0000310A00D5C
:100600002008D9044B080139A000A00DA00DA00DB1
:10061000F830A00520085904D800490808390038E6
:10062000031D581658081F39B500640064004C08B3
:100630008039D900D90ED90CD90CD90C0130D90583
:100640004C084039A000A00EA00C0730A0052008DF
:10065000D9044C082039A000A00CA00CA00C1F301D
:10066000A0052008D9044C081039A0000310A00CE4
:1006700020085904D8004C0801390038031D5816C9
:1006800058081F39B60064004D080839D900D90C44
:10069000D90CD90C1F30D9054D080439A00003101E
:1006A000A00C2008D9044D080239A0000310A00DA9
:1006B0002008D9044D080139A000A00DA00DA00DFF
:1006C000F830A00520085904D8004C080239003839
:1006D000031D581658081F39B70064004D088039AB
:1006E000D900D90ED90CD90CD90C0130D9054D0837
:1006F0004039A000A00EA00C0730A0052008D904A6
:100700004D082039A000A00CA00CA00C1F30A005A3
:100710002008D9044D081039A0000310A00C2008AF
:100720005904D8004C0804390038031D58165808DD
:100730001F39B80064004E080839D900D90CD90C0B
:10074000D90C1F30D9054E080439A0000310A00CA5
:100750002008D9044E080239A0000310A00D20087B
:10076000D9044E080139A000A00DA00DA00DF8304D
:10077000A00520085904D8004C0808390038031D8A
:0C078000581658081F39B900B929630049
:02400E00FE3F73
:00000001FF
